:100000000C9438000C9453000C9453000C9453003F
:100010000C9453000C9453000C94C2120C94530093
:100020000C9453000C9453000C9448130C94081334
:100030000C94560D0C9453000C9453000C945300E4
:100040000C9453000C9424020C9453000C94650CF3
:100050000C94B80C0C9453000C9453000C94530063
:100060000C9453000C9453000C9453000C945300C4
:1000700011241FBECFEFD4E0DEBFCDBF11E0A0E062
:10008000B1E0E6EAFEE202C005900D92A238B107A7
:10009000D9F713E0A2E8B1E001C01D92A939B10778
:1000A000E1F70C9460000C94000080E981BB8FE0C4
:1000B00084BBAC9AAD9A8EE28ABBD99ADD9A089538
:1000C0001F931092BC011092B8011092BD01A0E0E4
:1000D000B0E00E943F17802D992780938901A1E00D
:1000E000B0E00E943F17802D992780930001A2E085
:1000F000B0E00E943F17802D992780938A010E94CB
:1001000067120E9455000E9414028091890181307B
:1001100019F40E94500C02C00E94400C7894A89AD6
:100120000E94F1010E94C5060E94CD060E94D20FD6
:100130000E94EA060E942807809184018130C1F460
:10014000109284018091BC01882361F40E940C0DFF
:1001500080919C01882321F080910201823014F06B
:100160000E94C90D0E94490D0E944E0D0E9443102D
:10017000809188019091BC01813041F4992331F440
:100180000E94C20B0E94700F0E94CC0E80918701CA
:10019000813069F58091BC01882349F5AA9A0E94B3
:1001A000440B80919C01882369F40E945B130E9498
:1001B00097050E94FD040E94EC050E9479070E94A9
:1001C0009E0814C080910201823044F00E94EC0528
:1001D0000E9479070E949E080E945C07809102019C
:1001E000833024F00E9497050E94FD04AA98809114
:1001F00082018130B1F58091BC01882391F5109284
:10020000820180919C01882321F08091020183303A
:1002100014F00E9428078091990190919A0101960B
:1002200090939A01809399018091990190919A01FC
:10023000CC9769F4809197019091980101969093E1
:1002400098018093970110929A01109299010E944F
:1002500062090E94DD0680918F01813011F40E94B5
:10026000160A10918301113009F066CF8091BC010C
:10027000882309F061CF109283018091AD01813014
:1002800019F0823059F406C00E94740782E080930E
:10029000AD0104C00E9457071093AD0180919C01ED
:1002A000813009F049CF8091BC01882309F044CF07
:1002B00080919B01813009F03FCF10929B0180918A
:1002C0000201813071F082301CF4882339F034CF80
:1002D000823061F0833009F02FCF15C00E9474077F
:1002E0002BCF0E9457070E94920226CF0E945707E9
:1002F00064E084E00E948E010E94C5060E94CD0643
:100300000E94EA0619CF0E94570764E084E00E9429
:100310008E010E94C5060E94CD060ACF482FD998AB
:1003200027E030E0DB98000000000000000081E0E2
:1003300090E0022E02C0880F991F0A94E2F78423EE
:1003400011F0DA9A01C0DA98000000000000000005
:10035000DB9A0000000000000000215030408FEFC9
:100360002F3F3807F9F627E030E0DB980000000067
:100370000000000081E090E0022E02C0880F991F6B
:100380000A94E2F7862311F0DA9A01C0DA980000A5
:10039000000000000000DB9A0000000000000000E8
:1003A000215030408FEF2F3F3807F9F6DB98DA986D
:1003B000D99A089564E084E00E948E016CE480E0A4
:1003C0000E948E0110928401809184018823E1F3C0
:1003D0006AE08CE60E948E0160E085E00E948E015A
:1003E00008950E94DA01109282018091820188238F
:1003F000E1F30E94D5060E94920210928201809140
:1004000082018823E1F31092820180918201882386
:10041000E1F31092820164E084E00E948E016CE4BA
:1004200080E00E948E01089582E083BF92E49EBD29
:100430008EE189BF83E087BD86E982BD90938A0003
:1004400080E280937D0008951F920F920FB60F9265
:1004500011248F939F93809186018F5F80938601F3
:1004600080918601883439F591E09093850110924E
:100470008601809191038F5F809391038091910316
:10048000843631F41092910390938201909383010A
:1004900080919103823311F49093830180919003B2
:1004A0008F5F80939003809190038A3021F41092A3
:1004B0009003909384019F918F910F900FBE0F90A6
:1004C0001F901895282F80538A3010F090E005C0B7
:1004D000203311F49AE001C0982F822F81548A3181
:1004E00010F4922F9653822F81568A3110F4922F56
:1004F0009C532D3211F499E403C02E3209F491E497
:10050000892F992787FD909508958D3211F489E4FC
:1005100005C0803311F48AE001C08053992787FD1C
:100520009095089560E085E00E948E0163E886E082
:100530000E948E0160E987E00E948E0160E085E004
:100540000E948E0164E886E00E948E0161E987E0E6
:100550000E948E0160E085E00E948E0165E886E0E1
:100560000E948E0162E987E00E948E0160E085E0D2
:100570000E948E0166E886E00E948E0163E987E0B2
:100580000E948E0160E085E00E948E0167E886E0AF
:100590000E948E0164E987E00E948E0160E085E0A0
:1005A0000E948E0168E886E00E948E0165E987E07E
:1005B0000E948E0160E085E00E948E0169E886E07D
:1005C0000E948E0166E987E00E948E0160E085E06E
:1005D0000E948E016AE886E00E948E0167E987E04A
:1005E0000E948E0160E085E00E948E0161EA86E053
:1005F0000E948E0168E987E00E948E0160E085E03C
:100600000E948E0162EA86E00E948E0169E987E01D
:100610000E948E0160E085E00E948E0163EA86E020
:100620000E948E016AE987E00E948E0160E085E009
:100630000E948E0164EA86E00E948E016BE987E0E9
:100640000E948E0160E085E00E948E0165EA86E0EE
:100650000E948E016CE987E00E948E0160E085E0D7
:100660000E948E0166EA86E00E948E016DE987E0B5
:100670000E948E0160E085E00E948E0167EA86E0BC
:100680000E948E016EE987E00E948E0160E085E0A5
:100690000E948E0168EA86E00E948E016FE987E081
:1006A0000E948E0160E085E00E948E016FEB86E083
:1006B0000E948E0160EA87E00E948E0160E085E082
:1006C0000E948E0160EC86E00E948E0161EA87E064
:1006D0000E948E0160E085E00E948E0161EC86E060
:1006E0000E948E0162EA87E00E948E0160E085E050
:1006F0000E948E0162EC86E00E948E0163EA87E030
:100700000E948E0160E085E00E948E0163EC86E02D
:100710000E948E0164EA87E00E948E0160E085E01D
:100720000E948E0164EC86E00E948E0165EA87E0FB
:100730000E948E0160E085E00E948E0165EC86E0FB
:100740000E948E0166EA87E00E948E0160E085E0EB
:100750000E948E0166EC86E00E948E0167EA87E0C7
:100760000E948E0160E085E00E948E016DED86E0C2
:100770000E948E0168EA87E00E948E0160E085E0B9
:100780000E948E016EED86E00E948E0169EA87E08C
:100790000E948E0160E085E00E948E016FED86E090
:1007A0000E948E016AEA87E00E948E0160E085E087
:1007B0000E948E0160EE86E00E948E016BEA87E067
:1007C0000E948E0160E085E00E948E0161EE86E06D
:1007D0000E948E016CEA87E00E948E0160E085E055
:1007E0000E948E0162EE86E00E948E016DEA87E033
:1007F0000E948E0160E085E00E948E0163EE86E03B
:100800000E948E016EEA87E00E948E0160E085E022
:100810000E948E0164EE86E00E948E016FEA87E0FE
:100820000E948E0160E085E00E948E016BEF86E001
:100830000E948E0160EB87E00E948E0160E085E0FF
:100840000E948E016CEF86E00E948E0161EB87E0D2
:100850000E948E0160E085E00E948E016DEF86E0CF
:100860000E948E0162EB87E00E948E0160E085E0CD
:100870000E948E016EEF86E00E948E0163EB87E09E
:100880000E948E0160E085E00E948E016FEF86E09D
:100890000E948E0164EB87E00E948E0161E085E09A
:1008A0000E948E0160E086E00E948E0165EB87E089
:1008B0000E948E0161E085E00E948E0161E086E089
:1008C0000E948E0166EB87E00E948E010895CF9210
:1008D000DF92EF92FF920F931F93CF93DF936C0100
:1008E000062FEC0115C06D2F772785E00E948E0141
:1008F0006C2F86E00E948E01F701EE0FFF1FEE0DB8
:10090000FF1DE05EFE4F608187E00E948E01219610
:10091000C6010996E02EFF24C817D90720F38601E7
:100920000C5F1F4F612F772785E00E948E01602F9B
:1009300086E00E948E01E701CC0FDD1FCE0DDF1D8A
:10094000C05EDE4F698187E00E948E018A81882324
:1009500081F086010E5D1F4F612F772785E00E9491
:100960008E01602F86E00E948E016A8187E00E94DE
:100970008E01DF91CF911F910F91FF90EF90DF904B
:10098000CF9008950F931F93CF93DF938C01EC01C9
:100990000EC06D2F772785E00E948E016C2F86E0B8
:1009A0000E948E0160E087E00E948E012196C801BE
:1009B0000996C817D90768F38091AB019927FC0104
:1009C000EE0FFF1FE80FF91FE05EFE4F82818823C4
:1009D00079F00E5D1F4F612F772785E00E948E0111
:1009E000602F86E00E948E0160E087E00E948E0109
:1009F000DF91CF911F910F9108951F93CF93DF93B4
:100A000080914C0390914D0366E170E00E94F516D1
:100A10009B0177FD1BC0CB016AE070E00E94F516D8
:100A2000182F1695C9016AE070E00E94F51687E05C
:100A300090E0861B91092EE130E0829FE001839FC8
:100A4000D00D929FD00D11242A9616C03095219575
:100A50003F4FC9016AE070E00E94F516182F169505
:100A60001C5FC9016AE070E00E94F5168EE1689F84
:100A7000E0011124C650DF4F80911C0190911D01AF
:100A8000C817D90739F080911C0190911D010E946F
:100A9000C20404C08091AB01811721F0612FCE0107
:100AA0000E9467041093AB01D0931D01C0931C01F9
:100AB000DF91CF911F9108950F931F93CF93DF93F1
:100AC000EC01062F10E06D2F772785E00E948E0144
:100AD0006C2F86E00E948E01E02FFF27E25CFE4F24
:100AE000608187E00E948E016E96125E103F59F77A
:100AF000DF91CF911F910F9108951F93CF93DF93B3
:100B0000EC0110E06D2F772785E00E948E016C2F9D
:100B100086E00E948E0160E087E00E948E016E9662
:100B2000125E103F79F7DF91CF911F9108951F93C7
:100B3000CF93DF9380914E0390914F0366E170E075
:100B40000E94F5169B012A5F3F4F37FD12C0C90175
:100B50006AE070E00E94F516182F16951C5FC90117
:100B60006AE070E00E94F516C6E8D0E0C61BD10925
:100B700013C0309521953F4FC9016AE070E00E9493
:100B8000F516182F1695C9016AE070E00E94F51657
:100B9000C62FDD27C957DF4F80911E0190911F019D
:100BA000C817D90739F080911E0190911F010E944A
:100BB0007D0504C08091AC01811721F0612FCE0129
:100BC0000E945C051093AC01D0931F01C0931E01DD
:100BD000DF91CF911F910895FF920F931F93CF93B1
:100BE000DF9380915E0390915F038E55904063E0A8
:100BF00070E00E94F516EB016A3071051CF0C9E047
:100C0000D0E004C077FF02C0C0E0D0E08091950141
:100C100090919601C817D90709F47DC0C230D1055B
:100C200014F468E101C068E084E00E948E01D09372
:100C30009601C0939501C530D105B9F1C630D105F3
:100C40007CF4C230D10521F1C330D1051CF42197C9
:100C5000A9F419C0C330D10501F1249779F421C05A
:100C6000C730D10549F1C730D1051CF1C830D105D5
:100C700031F1299719F45BE8F52E23C048E8F42EEA
:100C800004E810E820C038E8F32E04E811E81BC09F
:100C900028E8F22E04E812E816C098E8F92E04E8D5
:100CA00011C088E8F82E05E80DC008E8F02E06E827
:100CB00009C018E8F12E05C0B9E8FB2E02C0AAE869
:100CC000FA2E07E813E860E085E00E948E0160E2FA
:100CD00086E00E948E01612F87E00E948E0160E015
:100CE00085E00E948E016EE386E00E948E01602FF7
:100CF00087E00E948E0160E085E00E948E016CE535
:100D000086E00E948E016F2D87E00E948E0160E0D8
:100D100084E00E948E01DF91CF911F910F91FF908F
:100D20000895EF92FF920F931F93CF93DF937A0171
:100D30009EE1699FB0011124680F711D8B01020FA4
:100D4000111D10929203EB0116C06D2F772785E0DD
:100D50000E948E016C2F86E00E948E01809192038A
:100D6000F701E80FF11D60818F5F8093920387E0A8
:100D70000E948E012196C017D10738F3DF91CF91E1
:100D80001F910F91FF90EF90089524E043E051E010
:100D90006EE088E10E949106089525E047E051E069
:100DA0006EE082E00E949106089520E14CE051E05F
:100DB00062E087E00E949106089580918A01813067
:100DC00041F42091C50146EC51E061E08AE00E94C7
:100DD0009106089560E085E00E948E0160E286E061
:100DE0000E948E0160E887E00E948E0160E085E04D
:100DF0000E948E016EE386E00E948E0164E887E027
:100E00000E948E0160E085E00E948E016CE586E024
:100E10000E948E0168E887E00E948E01089560E0DC
:100E200085E00E948E016FEC86E00E948E016CE8E6
:100E300087E00E948E0161E085E00E948E016BE0F8
:100E400086E00E948E016DE887E00E948E01089581
:100E500089ED8093920360E085E00E948E016091AD
:100E6000920386E00E948E0164E587E00E948E0175
:100E7000809192038F5F809392038C3D60F385EEA7
:100E80008093920360E085E00E948E01609192035E
:100E900086E00E948E0164E587E00E948E018091C9
:100EA00092038F5F80939203883E60F308956CE411
:100EB00080E00E948E01089580916003909161030B
:100EC000843B910544F48091AD01882361F481E075
:100ED0008093AD0108958091AD01181614F40E941D
:100EE00057071092AD01089562E480E00E948E01E0
:100EF0000895EF92FF920F931F93CF93DF93CDB797
:100F0000DEB72D970FB6F894DEBF0FBECDBFDE0162
:100F10001196E8E4F1E083E001900D928150E1F751
:100F200080915603909157036EE170E00E94F51690
:100F30008E01075F1F4FCB0177FF02C080E090E07A
:100F40004AE050E0B8010E94B016F801019000207C
:100F5000E9F73197EE2EE01A10929203FF240AC0AF
:100F60000E0F1F1FEC0FFD1F81850E946202F8010A
:100F70008083F394EF2DFF278E2D992787FD909581
:100F80008E010C5F1F4FE817F90754F3F09292039C
:100F900023E0AE014F5F5F4F6EE088E10E94910653
:100FA0002E2DA8016EE08BE18E190E9491062D96E0
:100FB0000FB6F894DEBF0FBECDBFDF91CF911F916A
:100FC0000F91FF90EF900895EF92FF920F931F9370
:100FD000CF93DF93CDB7DEB72F970FB6F894DEBF70
:100FE0000FBECDBF85E0FE01369611928A95E9F7D6
:100FF0008091A5019091A6018E01055F1F4F4AE0E7
:1010000050E0B8010E94B016F80101900020E9F705
:101010003197EE2EE01A10929203FF240AC00E0FB1
:101020001F1FEC0FFD1F83850E946202F801808361
:10103000F394EF2DFF278E2D992787FD90958E0134
:101040000F5F1F4FE817F90754F3F092920324E063
:10105000AE014A5F5F4F67E089E10E9491062E2D45
:10106000A80167E08CE18E190E9491068091A5018C
:101070009091A60118161906C4F460E085E00E945C
:101080008E016FEC86E00E948E016CE887E00E9482
:101090008E0161E085E00E948E016BE086E00E9497
:1010A0008E0160E087E00E948E018091A501909101
:1010B000A60197FF18C060E085E00E948E016FECEA
:1010C00086E00E948E0160E087E00E948E0161E070
:1010D00085E00E948E016BE086E00E948E016DE843
:1010E00087E00E948E018091A5019091A601892B35
:1010F000C1F460E085E00E948E016FEC86E00E9402
:101100008E0160E087E00E948E0161E085E00E9430
:101110008E016BE086E00E948E0160E087E00E9415
:101120008E012F960FB6F894DEBF0FBECDBFDF91B4
:10113000CF911F910F91FF90EF900895EF92FF9242
:101140000F931F93CF93DF93CDB7DEB72B970FB6D7
:10115000F894DEBF0FBECDBFDE011196EBE4F1E0E7
:1011600083E001900D928150E1F78E01085F1F4FDF
:101170004AE050E0B80180915C0390915D030E94C9
:10118000B016F80101900020E9F73197EE2EE01A31
:1011900010929203FF240AC00E0F1F1FEC0FFD1FB9
:1011A00080850E946202F8018083F394EF2DFF276F
:1011B0008E2D992787FD90958E010C5F1F4FE817A4
:1011C000F90754F3F092920323E0AE014F5F5F4FB3
:1011D0006EE08DE00E9491062E2DA8016EE080E168
:1011E0008E190E9491062B960FB6F894DEBF0FBEA3
:1011F000CDBFDF91CF911F910F91FF90EF90089598
:10120000EF92FF920F931F93CF93DF93CDB7DEB78B
:101210002B970FB6F894DEBF0FBECDBFDE0111963F
:10122000EEE4F1E083E001900D928150E1F78E0150
:10123000085F1F4F4AE050E0B8018091620390912F
:1012400063030E94B016F80101900020E9F731977E
:10125000EE2EE01A10929203FF240AC00E0F1F1FF9
:10126000EC0FFD1F80850E946202F8018083F394D9
:10127000EF2DFF278E2D992787FD90958E010C5F0E
:101280001F4FE817F90754F3F092920323E0AE01E1
:101290004F5F5F4F6DE08DE00E9491062E2DA801FB
:1012A0006DE080E18E190E9491062B960FB6F8949E
:1012B000DEBF0FBECDBFDF91CF911F910F91FF9089
:1012C000EF900895EF92FF920F931F93CF93DF93C8
:1012D000CDB7DEB728970FB6F894DEBF0FBECDBFEF
:1012E00019828AE08A8380919701909198018E01FA
:1012F0000A5F1F4F4AE050E0B8010E94B016F801A3
:1013000001900020E9F73197EE2EE01A1092920337
:10131000FF240DC08E010D5F1F4F0E0F1F1FEC0F1E
:10132000FD1F86810E946202F8018083F394EF2DF5
:10133000FF278E2D992787FD9095E817F90754F31D
:10134000F092920380919701909198018E010D5F28
:101350001F4F0A976CF421E0AE014F5F5F4F6EE0C4
:1013600082E00E94910621E0A8016EE083E004C0C3
:1013700022E0A8016EE082E00E949106809199012E
:1013800090919A018E010A5F1F4F4AE050E0B80128
:101390000E94B016F80101900020E9F73197EE2E77
:1013A000E01A10929203FF240DC08E010D5F1F4FB3
:1013B0000E0F1F1FEC0FFD1F86810E946202F801B5
:1013C0008083F394EF2DFF278E2D992787FD90952D
:1013D000E817F90754F3F0929203809199019091E4
:1013E0009A018E010D5F1F4F0A976CF421E0AE0148
:1013F0004E5F5F4F6EE085E00E94910621E0A801FC
:101400006EE086E004C022E0A8016EE085E00E9464
:10141000910628960FB6F894DEBF0FBECDBFDF91C0
:10142000CF911F910F91FF90EF900895CF92DF928F
:10143000EF92FF920F931F93CF93DF93CDB7DEB759
:101440002B970FB6F894DEBF0FBECDBF80919001F1
:101450009091910162E070E00E94F5167093910105
:1014600060939001809190019091910184569040F9
:1014700090939101809390018091900190919101BE
:1014800097FF04C0109291011092900180919001F9
:10149000909191018D5A964234F08CEA96E29093A5
:1014A000910180939001809190019091910164E667
:1014B00070E00E94E11670938C0160938B01809123
:1014C00090019091910164E670E00E94E116909382
:1014D0008E0180938D0180918D0190918E016AE043
:1014E00070E00E94E11670938E0160938D018091EF
:1014F0008B0190918C0125E429831A821B828E0135
:10150000085F1F4F4AE050E0B8010E94B016F80192
:1015100001900020E9F73197CE2EC01A1092920365
:10152000DD240BC0020F131FE20EF31EF7018081B2
:101530000E946202F8018083D3942D2D33278C2DD5
:10154000992787FD909578E0E72EF12CEC0EFD1E93
:101550008E010C5F1F4F2817390724F3D092920396
:1015600022E0AE014E5F5F4F63E084E00E9491068F
:101570002C2DA80163E086E08C190E9491068091D1
:101580008D0190918E014AE050E0B7010E94B016A3
:10159000F70101900020E9F73197EE19EE2E109235
:1015A0009203FF240AC00E0F1F1FEC0FFD1F808542
:1015B0000E946202F8018083F394EF2DFF278E2DA5
:1015C000992787FD90958E010C5F1F4FE817F9074B
:1015D00054F3F092920321E0AE014F5F5F4F63E05E
:1015E00086E00E94910621E0AE014E5F5F4F63E00E
:1015F00087E00E94910621E0A80163E087E00E9455
:1016000091062B960FB6F894DEBF0FBECDBFDF91CB
:10161000CF911F910F91FF90EF90DF90CF900895A1
:101620000F931F93CF93DF93CDB7DEB72A970FB6F3
:10163000F894DEBF0FBECDBF4AE050E08E010F5FD1
:101640001F4FB8010E94B016F80101900020E9F781
:101650003197E01B1092920320E0FF27E7FDF09501
:1016600001C02F5F822F99278E179F07D4F32093F5
:1016700092032A960FB6F894DEBF0FBECDBFDF915E
:10168000CF911F910F910895EF92FF920F931F93A7
:10169000CF93DF938091B602843409F06AC033E0BF
:1016A000E32EF12C60E070E0A7EBB2E08C91FD013D
:1016B000218112810381E70124967E011496613411
:1016C000710509F456C0422F55274D535040E09103
:1016D0005101F0915201E60FF71F9927CD97880F1E
:1016E000991F880F991F9A01689413F835952795CB
:1016F0001694E1F7822B932B808360347105C9F136
:10170000212F33272D533040FB0131968091510119
:1017100090915201E80FF91F4F70507084E0440F10
:10172000551F8A95E1F7C9019595879595958795F8
:10173000482B592B4083CB35D105D9F0FB0132968C
:101740008091510190915201E80FF91F2370307080
:1017500086E0220F331F8A95E1F7802F9927CD97D6
:10176000282B392B20836E33710519F06D5F7F4F65
:101770009DCF10928701DF91CF911F910F91FF9024
:10178000EF900895EF92FF920F931F93CF93DF9303
:101790008091DC01843409F06AC033E0E32EF12C3F
:1017A00060E070E0ADEDB1E08C91FD01218112812E
:1017B0000381E70124967E0114966134710509F4D2
:1017C00056C0422F55274D535040E0915301F091A0
:1017D0005401E60FF71F9927CD97880F991F880F9F
:1017E000991F9A01689413F8359527951694E1F797
:1017F000822B932B808360347105C9F1212F33270D
:101800002D533040FB01319680915301909154014A
:10181000E80FF91F4F70507084E0440F551F8A95F0
:10182000E1F7C9019595879595958795482B592B93
:101830004083CB35D105D9F0FB013296809153011D
:1018400090915401E80FF91F2370307046E0220F89
:10185000331F4A95E1F7802F9927CD97282B392BF5
:1018600020836E33710519F06D5F7F4F9DCF10920D
:101870008801DF91CF911F910F91FF90EF90089514
:1018800082E289B910BC80B91CBE909A28E92AB9B5
:1018900096E890BD82EC8BB921B99CBF82B90895BE
:1018A00082E289B910BC80B91CBE909A88E98AB9D5
:1018B00026E820BD92EC9BB980E981B92CBF92B992
:1018C0000895159BFECF83B908951F920F920FB60E
:1018D0000F9211248F939F93EF93FF939CB190935A
:1018E00093039D3081F48091AF01813061F4AB9816
:1018F0001092AF0180938801E0918F03FF27E65299
:10190000FE4F90832CC08091AF01882319F0813065
:1019100031F513C0933239F480918801882319F48A
:1019200081E08093AF0110928F0380918F03E82FA5
:10193000FF27E652FE4F90830CC0E0918F03FF27F4
:10194000E652FE4F908380918F03853930F4809169
:101950008F038F5F80938F0302C01092AF01FF91BE
:10196000EF919F918F910F900FBE0F901F90189540
:101970001F920F920FB60F9211248F939F93EF93A4
:10198000FF9393B1909394039D3081F48091AE01C5
:10199000813061F4AB981092AE0180938701E091A1
:1019A0008C03FF27EC54FD4F90832DC08091AE0136
:1019B000882319F0813039F514C0933241F48091B5
:1019C0008701882321F481E08093AE01AB9A1092C5
:1019D0008C0380918C03E82FFF27EC54FD4F9083FC
:1019E0000CC0E0918C03FF27EC54FD4F9083809155
:1019F0008C03853930F480918C038F5F80938C0346
:101A000002C01092AE01FF91EF919F918F910F90C4
:101A10000FBE0F901F901895CF93DF93CDB7DEB711
:101A20002A970FB6F894DEBF0FBECDBF83E289833D
:101A30001A8283E68B831C821D8286E890E060E038
:101A400070E10E94F5169C0160E470E00E94F516BA
:101A5000635C6E83C90160E470E00E94F516835CEC
:101A60008F838DE08887FE0131969E01275F3F4F6F
:101A70008081159BFECF83B93196E217F307C1F73A
:101A80002A960FB6F894DEBF0FBECDBFDF91CF917F
:101A9000089585B392E0892785BB089590919401BC
:101AA000913019F485B3892785BB08951F920F9251
:101AB0000FB60F9211242F933F935F936F937F93F1
:101AC0008F939F93AF93BF938091B0019091B10199
:101AD000892B81F484B595B59093B7018093B601B5
:101AE0008EB58F7B8EBD81E090E09093B1018093A5
:101AF000B00141C084B595B59093B5018093B40110
:101B00002EB520642EBD2091B6013091B701821B05
:101B1000930B1092B1011092B001865698406CE27E
:101B200071E00E94E1167093B3016093B20177FFF8
:101B300005C01092B3011092B20109C0673071055F
:101B400034F086E090E09093B3018093B20120914D
:101B5000B2013091B30180910201992787FD9095E0
:101B60002817390741F0263031052CF42093020163
:101B700081E080939B01BF91AF919F918F917F9165
:101B80006F915F913F912F910F900FBE0F901F901B
:101B90001895809156039091570390939E018093DE
:101BA0009D0180919D0190919E0120919F01309116
:101BB000A001821B930B9093A2018093A1018091BD
:101BC0009D0190919E019093A00180939F0180912F
:101BD000A3019091A4012091A1013091A201820F53
:101BE000931F9093A4018093A3018091A701843057
:101BF000F1F41092A7016091A3017091A4018827CC
:101C000077FD8095982F0E94361420E030E040EC5C
:101C10005FE30E947C130E949F147093A60160935F
:101C2000A5011092A4011092A3010E94E4078091E3
:101C3000A7018F5F8093A7010895BF92CF92DF9293
:101C4000EF92FF920F931F93CF93DF93CDB7DEB741
:101C500060970FB6F894DEBF0FBECDBF19821A820F
:101C60001B821C828091A8029091A90290939803F4
:101C7000809397038091AA029091AB029093960370
:101C80008093950380919703909198038E01055F4F
:101C90001F4F4AE050E0B8010E94B016F8010190D1
:101CA0000020E9F73197BE2EB01ACC24DD240DC0F8
:101CB000EC0CFD1CF70180810E9462020C0D1D1DC1
:101CC000F80180830894C11CD11C8B2D992787FDB6
:101CD00090952BE0E22EF12CEC0EFD1E8E010B5F99
:101CE0001F4FC816D90624F324E0AE014F5F5F4FA3
:101CF00061E08CE00E9491062B2DA80161E080E15B
:101D00008B190E94910680919503909196034AE069
:101D100050E0B7010E94B016F70101900020E9F7EA
:101D20003197DE2EDE18EE24FF240DC0FE01EE0DED
:101D3000FF1D83850E9462020E0D1F1DF801808326
:101D40000894E11CF11C8D2D992787FD90958E013B
:101D50000B5F1F4FE816F9064CF324E0AE014F5F0E
:101D60005F4F62E08CE00E9491062D2DA80162E099
:101D700080E18D190E94910660960FB6F894DEBF3F
:101D80000FBECDBFDF91CF911F910F91FF90EF90CC
:101D9000DF90CF90BF9008958F929F92BF92CF9285
:101DA000DF92EF92FF920F931F93CF93DF93CDB704
:101DB000DEB760970FB6F894DEBF0FBECDBF1982B5
:101DC0001A821B821C8280907003909071038E0196
:101DD000055F1F4F4AE050E0B80180916E0390917B
:101DE0006F030E94B016F80101900020E9F73197C7
:101DF000BE2EB01ACC24DD240DC0EC0CFD1CF70166
:101E000080810E9462020C0D1D1DF80180830894E0
:101E1000C11CD11C8B2D992787FD90953BE0E32EAB
:101E2000F12CEC0EFD1E8E010B5F1F4FC816D9065C
:101E300024F324E0AE014F5F5F4F64E08CE00E942A
:101E400091062B2DA80164E080E18B190E94910678
:101E50004AE050E0B701C4010E94B016F7010190BA
:101E60000020E9F73197DE2EDE18EE24FF240DC0A6
:101E7000FE01EE0DFF1D83850E9462020E0D1F1DE7
:101E8000F80180830894E11CF11C8D2D992787FDB2
:101E900090958E010B5F1F4FE816F9064CF324E076
:101EA000AE014F5F5F4F65E08CE00E9491062D2DE3
:101EB000A80165E080E18D190E94910660960FB639
:101EC000F894DEBF0FBECDBFDF91CF911F910F9170
:101ED000FF90EF90DF90CF90BF909F908F900895EC
:101EE000DF92EF92FF920F931F93CF93DF93CDB7C3
:101EF000DEB72B970FB6F894DEBF0FBECDBFDE0165
:101F00001196E9E5F1E083E001900D928150E1F74F
:101F10008E01085F1F4F4AE050E0B8018091B00287
:101F20009091B1020E94B016F80101900020E9F7EB
:101F30003197DE2ED01AEE24FF240DC0FE01EE0DE7
:101F4000FF1D80850E9462020E0D1F1DF801808317
:101F50000894E11CF11C8D2D992787FD90958E0129
:101F60000C5F1F4FE816F9064CF323E0AE014F5FFC
:101F70005F4F61E088E10E9491062D2DA80161E08C
:101F80008BE18D190E9491062B960FB6F894DEBF57
:101F90000FBECDBFDF91CF911F910F91FF90EF90BA
:101FA000DF90089522E047E551E061E08AE10E9478
:101FB00091060895F89488E190E028E00FB6F8942F
:101FC000A89581BD0FBE21BDFFCF64E084E00E94D3
:101FD0008E012091C50146EC51E062E08AE00E944A
:101FE000910668E084E00E948E0126E04CE551E015
:101FF00065E08AE00E94910680910001813021F421
:1020000023E044E751E003C023E047E751E065E007
:1020100081E10E94910660E084E00E948E0126E04A
:1020200042E651E066E08AE00E94910680918901D3
:10203000813021F423E044E751E003C023E047E787
:1020400051E066E081E10E94910626E048E651E019
:1020500067E08AE00E94910680918A01813021F434
:1020600023E044E751E003C023E047E751E067E0A5
:1020700081E10E94910626E04EE651E068E08AE0A8
:102080000E94910608959D998EC08091B8018F5F3E
:102090008093B80191E09093BA018091B8018530A6
:1020A00009F085C08091BC01882339F49093BC016C
:1020B0001092BD010E94E50F78C09091BD01913052
:1020C00071F580918901882319F49093890102C0E8
:1020D0001092890180918901A0E0B0E0082E0E9451
:1020E000471768E084E00E948E0126E042E651E056
:1020F00066E08AE00E94910680918901813021F496
:1021000023E044E751E003C023E047E751E066E005
:1021100081E10E94910660E084E00E948E0180913E
:10212000BD01823079F580918A01882321F481E014
:1021300080938A0102C010928A0180918A01A2E0F4
:10214000B0E0082E0E94471768E084E00E948E01EC
:1021500026E048E651E067E08AE00E94910680911F
:102160008A01813021F423E044E751E003C023E0F9
:1021700047E751E067E081E10E94910660E084E07A
:102180000E948E018091BD01833089F41092BC01C0
:10219000F89488E190E028E00FB6F894A89581BD06
:1021A0000FBE21BDFFCF1092B8011092BA019C99C9
:1021B0007FC19091BC01913009F080C19093BB0127
:1021C0008091B9018F5F8093B9018091B901853009
:1021D00009F074C11092B9018091BD01813009F4F8
:1021E0004CC0813038F0823009F4A1C0833009F04E
:1021F00065C1FEC09093BD0164E084E00E948E0141
:102200002091C50146EC51E062E08AE00E9491060F
:1022100026E04CE551E065E08AE00E94910680915D
:102220000001813021F423E044E751E003C023E0C2
:1022300047E751E065E081E10E94910668E084E0B3
:102240000E948E0126E042E651E066E08AE00E94AC
:10225000910680918901813021F423E044E751E027
:1022600003C023E047E751E066E081E10E94910668
:1022700060E084E00E948E01FDC082E08093BD0199
:1022800064E084E00E948E012091C50146EC51E09B
:1022900062E08AE00E94910626E04CE551E065E0AC
:1022A0008AE00E94910680910001813021F423E0B0
:1022B00044E751E003C023E047E751E065E081E1F6
:1022C0000E94910626E042E651E066E08AE00E9424
:1022D000910680918901813021F423E044E751E0A7
:1022E00003C023E047E751E066E081E10E949106E8
:1022F00068E084E00E948E0126E048E651E067E055
:102300008AE00E94910680918A01813021F423E0C5
:1023100044E751E003C023E047E751E067E081E193
:102320000E94910660E084E00E948E01B9C083E0C3
:102330008093BD0164E084E00E948E012091C5017C
:1023400046EC51E062E08AE00E94910626E04CE50E
:1023500051E065E08AE00E949106809100018130A1
:1023600021F423E044E751E003C023E047E751E0D4
:1023700065E081E10E94910626E042E651E066E0D8
:102380008AE00E94910680918901813021F423E046
:1023900044E751E003C023E047E751E066E081E114
:1023A0000E94910626E048E651E067E08AE00E943C
:1023B000910680918A01813021F423E044E751E0C5
:1023C00003C023E047E751E067E081E10E94910606
:1023D00068E084E00E948E0126E04EE651E068E06D
:1023E0008AE00E94910660E084E00E948E010895D8
:1023F0001092BD0164E084E00E948E012091C5012D
:1024000046EC51E062E08AE00E94910668E084E0D8
:102410000E948E0126E04CE551E065E08AE00E94D2
:10242000910680910001813021F423E044E751E0DE
:1024300003C023E047E751E065E081E10E94910697
:1024400060E084E00E948E0126E042E651E066E012
:102450008AE00E94910680918901813021F423E075
:1024600044E751E003C023E047E751E066E081E143
:102470000E94910626E048E651E067E08AE00E946B
:10248000910680918A01813021F423E044E751E0F4
:1024900003C023E047E751E067E081E10E94910635
:1024A00026E04EE651E068E08AE00E949106089539
:1024B0001092B9018091BA018091BB0108958130D9
:1024C00029F4A0E0B0E0062E0E9447170895EF928D
:1024D000FF920F931F93CF93DF93CDB7DEB764972F
:1024E0000FB6F894DEBF0FBECDBF40E050E08E01C6
:1024F0000F5F1F4F842F9927DC01AD5FBF4F0E94F4
:102500003F17202D3327F801E80FF91F20832223DE
:10251000F1F04F5F5F4F2F3F69F7108218C0FE0147
:10252000E00FF11F81810E9462020A531E4FF801E1
:1025300080830E2D11278091C5010894E11CF11CA8
:10254000992787FD9095081719074CF30EC0DE01F7
:102550001196FD0101900020E9F73197EA1BFB0B72
:10256000E093C501EE24FF24E4CF64960FB6F894FF
:10257000DEBF0FBECDBFDF91CF911F910F91FF90B6
:10258000EF9008951F920F920FB60F9211242F9380
:102590003F938F939F9321E020938F018091BE0101
:1025A000882381F480918000909181009093C001F4
:1025B0008093BF0180918A008F7B80938A00209353
:1025C000BE011DC080918000909181009093910187
:1025D0008093900180918A00806480938A00109299
:1025E000BE0180919001909191012091BF013091A5
:1025F000C001821B930B90939101809390019F9156
:102600008F913F912F910F900FBE0F901F901895B3
:102610001F920F920FB60F9211248F939F93809168
:10262000C4018130A9F0813018F0823051F526C004
:102630008091C2018E3131F41092C20181E0809309
:10264000C401979A8091C2018F5F8093C20119C023
:102650009091C301923061F41092C3018091C10145
:10266000813019F49093C40103C083E08093C401C6
:102670008091C3018F5F8093C30103C083E0809387
:10268000C4019F918F910F900FBE0F901F901895CE
:102690001F920F920FB60F9211248F938091C40155
:1026A000833019F41092C40197988F910F900FBE48
:1026B0000F901F90189580914C0390914D0365E009
:1026C00070E00E94F51666507F4F77FD0FC081E0E5
:1026D000653F78071CF064EF71E003C06B3F710544
:1026E0003CF06A5F81E08093C10104C060E070E06B
:1026F0001092C10162BD0895A8E1B0E0E2E8F3E103
:102700000C940E1769837A838B839C832D833E837D
:102710004F835887B1E18B2E912C8C0E9D1EB401F6
:10272000CE0101960E9411168E01075F1F4FB8015E
:10273000CE0105960E9411162989223008F46AC03C
:102740003985323008F468C08A899A8589278A8B4E
:10275000243009F463C0223009F460C0343041F4FD
:102760001D8A1E8A1F8A188E1C8A1B8AB40177C094
:10277000323009F458C06B897C898B859C85681B35
:10278000790B7C8B6B8B2D893E894F89588DED841D
:10279000FE840F8518892E153F054007510740F428
:1027A000220F331F441F551F615070407C8B6B8B71
:1027B00080E090E0A0E0B0E4AA24BB24650160E0E2
:1027C00070E02E153F054007510740F0A82AB92AAE
:1027D000CA2ADB2A2E193F09400B510BB695A79543
:1027E00097958795220F331F441F551F6F5F7F4FAB
:1027F0006F31710531F7D601C5018F779070A070E8
:10280000B07080349105A105B10589F0AD8ABE8A0A
:10281000CF8AD88EB40123C0B80121C03217D1F7B6
:102820006AE771E01CC084E0898BB40118C0A7FC82
:10283000EDCF211531054105510541F380E490E0CC
:10284000A0E0B0E0A80EB91ECA1EDB1E80E89FEF14
:10285000AFEFBFEFA822B922CA22DB22D7CFCB012C
:102860000E94EF14ECE068960C942A17A8E0B0E000
:10287000ECE3F4E10C9417179B01AC0183E089832E
:102880001A8257FD51C0211531054105510539F412
:1028900082E08983CE0101960E94EF144CC0EEE1E4
:1028A000F0E0FC83EB838A818823C9F1203010E0BB
:1028B000310710E0410710E85107C9F1882799272F
:1028C000DC01821B930BA40BB50B8D839E83AF831E
:1028D000B8872D813E814F815885203080E03807B0
:1028E00080E0480780E45807A8F6EB81FC81DA0114
:1028F000C901880F991FAA1FBB1F31979C01AD0109
:10290000803010E0910710E0A10710E4B10778F3E0
:10291000FC83EB838D839E83AF83B887BBCF2D83EE
:102920003E834F835887D5CF81E08A83ACCF60E068
:1029300070E080E09FECE3E028960C943317ACE065
:10294000B0E0E5EAF4E10C94181769837A838B838D
:102950009C83BE016B5F7F4FCE0101960E941116D2
:102960008D81823061F0823050F0843069F48E8144
:10297000882359F52FEF3FEF4FEF5FE72AC020E0A4
:1029800030E040E050E025C02F81388537FDF7CF9B
:102990002F31310564F78EE190E0821B930B29857E
:1029A0003A854B855C8504C05695479537952795A4
:1029B0008A95D2F78E81882361F0509540953095A5
:1029C00021953F4F4F4F5F4F04C020E030E040E083
:1029D00050E8CA01B901E2E02C960C9434174F92EA
:1029E0005F926F927F928F929F92AF92BF92DF928F
:1029F000EF92FF920F931F9320E030E040E050E011
:102A0000FC01E480F58006811781D18080818230CD
:102A100038F4D801C701A061AF77B0706FEFD9C0AB
:102A2000843009F46EC0823009F471C0E114F104FD
:102A30000105110509F46BC0828193816FEF823823
:102A400096070CF06AC062E87FEF681B790B6A3169
:102A500071050CF080C047015801062E04C0B694E1
:102A6000A794979487940A94D2F74424552432016A
:102A700081E090E0A0E0B0E004C0880F991FAA1F99
:102A8000BB1F6A95D2F70197A109B109E822F92283
:102A90000A231B23E114F1040105110529F061E06B
:102AA000462E512C612C712C85017401E428F528E7
:102AB00006291729D801C7018F779070A070B070D0
:102AC00080349105A105B10509F457C0D801C701AB
:102AD000CF96A11DB11D60E070E08030E0E09E0760
:102AE000E0E0AE07E0E4BE0710F061E070E027E050
:102AF000B695A795979587952A95D1F7AF77B0703A
:102B000068C080E090E0A0E0B0E06FEF62C080E0DD
:102B100090E0A0E0B0E060E05CC0803891058CF708
:102B2000BC0161587F4FD801C7018F779070A070AA
:102B3000B07080349105A105B105A1F08FE390E05C
:102B4000A0E0B0E0E80EF91E0A1F1B1F17FD28C009
:102B5000D801C701CCCF60E070E080E090E0A0E059
:102B6000B0E0CCCFE7FEF2CF80E490E0A0E0B0E0B0
:102B7000E80EF91E0A1F1B1FE9CFE7FC18C080E012
:102B800090E060E0E61660E0F60660E0060760E4CC
:102B9000160710F081E090E0BC01D801C701A7CF73
:102BA00016950795F794E7946F5F7F4FD1CFD801C3
:102BB000C701805C9F4FAF4FBF4F60E070E0803037
:102BC000E0E09E07E0E0AE07E0E4BE0708F48FCF48
:102BD0008CCF282F392F9A2F9F77842F8078892B9D
:102BE000962F9795992797958F77482F492B66951C
:102BF000852F8078862BD794DD24D7948F77582F14
:102C00005D29CA01B9011F910F91FF90EF90DF90EC
:102C1000BF90AF909F908F907F906F905F904F90FC
:102C20000895FC01DB01208131819281492F4F778A
:102C300050E0991F9927991F8381682F660F692B90
:102C4000881F8827881FFD018183662309F049C0FA
:102C5000211531054105510509F470C082E89FEF47
:102C6000FD0193838283220F331F441F551F220FC0
:102C7000331F441F551F220F331F441F551F220FA0
:102C8000331F441F551F220F331F441F551F220F90
:102C9000331F441F551F220F331F441F551F83E04E
:102CA0008C932030F0E03F07F0E04F07F0E45F073F
:102CB00090F482E89FEF220F331F441F551F0197A6
:102CC000203060E0360760E0460760E4560798F37E
:102CD000FD0193838283FD012483358346835783DB
:102CE00008956F3F71F1862F99278F579040FD010E
:102CF0009383828383E08C93220F331F441F551FDD
:102D0000220F331F441F551F220F331F441F551F0F
:102D1000220F331F441F551F220F331F441F551FFF
:102D2000220F331F441F551F220F331F441F551FEF
:102D300050642483358346835783089582E08C93BF
:102D40000895211531054105510519F484E08C934E
:102D5000089544FD02C01C92BECF81E08C93BBCF8E
:102D6000FB019F01E8944230C4F04532B4F44A308C
:102D700029F497FB1EF4909581959F4F642F772738
:102D80000E94E116805D8A330CF0895D8193CB014E
:102D90000097A1F716F45DE251931082C9010C94DB
:102DA000D116DC01FC0101900020E9F73297AE1743
:102DB000BF0730F47C916081708331976D93F7CFBA
:102DC0000895AA1BBB1B51E107C0AA1FBB1FA61772
:102DD000B70710F0A61BB70B881F991F5A95A9F7C4
:102DE00080959095BC01CD01089597FB092E07268B
:102DF0000AD077FD04D0E5DF06D000201AF47095E4
:102E000061957F4F0895F6F7909581959F4F0895AE
:102E10002F923F924F925F926F927F928F929F92EA
:102E2000AF92BF92CF92DF92EF92FF920F931F93D8
:102E3000CF93DF93CDB7DEB7CA1BDB0B0FB6F89489
:102E4000DEBF0FBECDBF09942A88398848885F84C9
:102E50006E847D848C849B84AA84B984C884DF803A
:102E6000EE80FD800C811B81AA81B981CE0FD11D1E
:102E70000FB6F894DEBF0FBECDBFED010895E19906
:102E8000FECFBFBBAEBBE09A11960DB20895E1999B
:102E9000FECFBFBBAEBB0DBA11960FB6F894E29A47
:062EA000E19A0FBE089547
:102EA60001010200000A3100004400005D5E5F4936
:102EB6005B1D5C00202936410A41072623002300BA
:102EC600546466536365526200516100506000505D
:102ED600600051610052620053636554646667681E
:102EE600696A6B6B6A696867000000000000000091
:102EF600004A0370020D0A0A1D0000001A0B160094
:102F060000001A0D470C1E001529323200000F3C36
:102F16002D380000191800192A2A000000000000A8
:022F26000000A9
:00000001FF
